:0A0000000216F8022FF75322C02267
:10000B0002309BD2B5D2B4220237FB244750524D5B
:07001B004300FAF9F8614609
:0700230002389A43EA402273
:07002B0002400175EAB0225A
:100033000258F4D2308B2C8A2D892E120072C0E024
:10004300FF121940D0E040F31214C3400122ECC068
:10005300E0EDC0E0EEC0E0EFC0E0120072D0F0AF20
:10006300F0D0F0AEF0D0F0ADF0D0F0ACF080D9E449
:1000730075F001782C120A1F020768C3EE6480949E
:100083008040028007C3E49FFFE49EFE2275A80020
:100093009000E27406F09000E07480F09000E27447
:1000A3000CF012203102046EE86480F8E933E8337F
:1000B30060110460F0ED33EC337009E8FCE9FDEA0C
:1000C300FEEBFF220460DED3EB9FEA9EE99DE8C2CC
:1000D300E78CF0C2F795F0400CE8CCF8E9CDF9EAEB
:1000E300CEFAEBCFFB12043985D0F058047003200D
:1000F300D5B3E80470075002B2D502047892D5EC68
:100103000460F7E4CCC0E0C398F8603B941860083F
:10011300400DD0E0FB020450E4FBFAC9FC8028E860
:1001230030E406E4C9FBE4CAFCE830E305E4C9CAE9
:10013300CBFCE854076010F8C3E913F9EA13FAEBB0
:1001430013FBEC13FCD8F130F52FC3E49CFCEF9BBD
:10015300FFEE9AFEED99FDD0E0FBEF4E4D4C701291
:1001630022DB03020475EC2CFCEF33FFEE33FEEDD0
:1001730033FDED30E7EB020450EF2BFFEE3AFEEDDB
:1001830039FDD0E0FB50130BBB0003020478ED13E1
:10019300FDEE13FEEF13FFEC13FC020450EC4D6075
:1001A30011E8497017ED33EC3304600DE4FCFFFEF6
:1001B300FD22E933E8330470F802046E120439585F
:1001C300046009E4CC2481500628500902047828ED
:1001D3004003020475C0E0EB4A7044B98006D0E0E6
:1001E300FB020464EF4E701CBD8008EBFFEAFEE9DE
:1001F300FD80EBE98DF0A4FEE5F0020289E9CDF97B
:10020300EAFEEBFFEF89F0A4FCE5F0CE89F0A42E23
:10021300FFE435F0CD89F0A42DFEE435F08067EFDF
:100223004E7005BD80D780C3EF8BF0A4ACF0EE8B8E
:10023300F0A42CFCE435F0F8EF8AF0A42CE5F038B8
:10024300FCE433CB8DF0A42CFCE5F03BF8EE8AF014
:10025300A42CFCE5F038F8E433CF89F0A42CFCE5BA
:10026300F038CF3400CE89F0A42FFFE5F03EFEE452
:1002730033C98DF0A42EFEE5F039CD8AF0A42FFF0B
:10028300E5F03EFEE43DFD33D0E0FB50070BBB0041
:100293000F020478EC2CFCEF33FFEE33FEED33FD5D
:1002A300020450020478EC5D046005E8590470030D
:1002B30002046E120439580460F6EC4860F2EC70E4
:1002C30004FDFEFF22C860DB2481C85009C3986087
:1002D3000250060204759850CAF582E9294B4A7008
:1002E30005AB8202046475F0007C1A7880C3EF9B2F
:1002F300EE9AED99400DC3EF9BFFEE9AFEED99FD4B
:10030300E842F0DC23ACF0D0E0FFD0E0FED0E0FD2B
:10031300AB8220E7101BEB60BAEC2CFCEF33FFEE53
:1003230033FEED33FD020450E803F830E705C0F077
:1003330075F000EF2FFFEE33FEED33FD40B830E7ED
:10034300C280AA74F8CC6480CCC86480C8F58204E7
:100353006043C3EB9FF5F0EA9E42F0E99D42F0E86B
:100363009C45F060305018E5825FFFE582F42B5521
:1003730082FB50210ABA001D09B90019088016E54D
:10038300825BFBE582F42F5582FF50090EBE000508
:100393000DBD00010CC3EB9FF5F0EA9E42F0E99D11
:1003A30042F0E89C45F06007CC4820E701B3EC221B
:1003B300ED33EC33600A047003BD8004ECB2E7FC58
:1003C3002275F020800E75F010800575F0087D0011
:1003D3007E007F003392D530D503120990EC334071
:1003E30010EF33FFEE33FEED33FDEC33FCD5F0EDD0
:1003F30022E5F0247EA2D513CC92E7CDCEFF22EDE9
:10040300D2E7CD33EC3392D524814006E4FFFEFDE1
:10041300FC22FCE4CFCECDCC24E0501174FF80ED60
:10042300C3CC13CCCD13CDCE13CECF13CF0470F0EA
:1004330030D5DE020990E9D2E7C933E833F892D523
:10044300EDD2E7CD33EC33FC5002B2D522EC30E7EA
:10045300100FBF000C0EBE00080DBD00040BEB60B7
:1004630014A2D5EB13FCED92E7FD2274FFFCFDFE15
:10047300FF22E480F8A2D574FF13FC7D80E480EFB3
:10048300F920E72824F950037907E4F42402FB1840
:10049300DBFDE624FB5014E9600DE4F618E604F6F0
:1004A300B40A08E4F6D9F57401F60A22C2D522ED9E
:1004B30033EC3392D5FA602AB4FF33EDC2E77BFF06
:1004C30060067A0479D7E4227A0479E020D5047AA5
:1004D3000479DB224E614E002B494E46002D494ED6
:1004E3004600E47A08F608DAFC7B00740722E8C0C9
:1004F300E0ECC0E0EDC0E0EEC0E0EFC0E0EA75F094
:1005030010A4CAABF075F04DA42BFBE435F0FCEA64
:100513002410FAEB34C5FBEC34D9FCEDC2E7FF75CC
:10052300F056A4F42411C5F0F434C58FF0A42AE5E1
:10053300F03BE43CF620E714120632D0E0FFD0E0B3
:10054300FED0E0FDD0E0FC1202A98014F4041206F0
:1005530032D0E0FFD0E0FED0E0FDD0E0FC1201A0FD
:10056300D0E0F8E6FAEDD2E7CD33EC332482FBE4B6
:10057300C3CF33CFCE33CECD33CD33DBF37B077550
:10058300F00A846004F6081B0AE5F0F6088FF0749D
:100593000AA4FFACF08EF0740AA42CFEACF0500158
:1005A3000C8DF0740AA42CFDE435F0F608DBDE7440
:1005B3000722C0E0EFFBEEFAEDF9ECF81201A0D050
:1005C300E0F5F0EFFBEEFAEDF9ECF81209CEA3A398
:1005D300A3A3E8C0E0E9C0E0EAC0E0EBC0E0C0F0FC
:1005E3001201A01209EBA3A3A3A31200AFD0F0D072
:1005F300E0FBD0E0FAD0E0F9D0E0F8D5F0D4223F28
:100603008000004120000042C80000447A000046F8
:100613001C400047C35000497424004B1896804C7B
:10062300BEBC205A0E1BCA6753C21C749DC5AEFBC9
:1006330060065407601C2323120660EB54386009DC
:1006430012064C12065B1201A0ECF8EDF9EEFAEF7C
:10065300CB22EB12065B80F1543803241C90060274
:10066300FE93FC0EEE93FD0EEE930ECE93FF22E768
:1006730009F608DFFA8046E709F208DFFA803E88C8
:10068300828C83E709F0A3DFFA8032E309F608DFFF
:10069300FA8078E309F208DFFA807088828C83E3BA
:1006A30009F0A3DFFA806489828A83E0A3F608DF76
:1006B300FA805889828A83E0A3F208DFFA804C80AB
:1006C300D280FA80C680D4806980F2803380108023
:1006D300A680EA809A80A880DA80E280CA80338983
:1006E300828A83ECFAE493A3C8C582C8CCC583CCC1
:1006F300F0A3C8C582C8CCC583CCDFE9DEE7800D93
:1007030089828A83E493A3F608DFF9ECFAA9F0ED72
:10071300FB2289828A83ECFAE0A3C8C582C8CCC5D0
:1007230083CCF0A3C8C582C8CCC583CCDFEADEE89E
:1007330080DB89828A83E493A3F208DFF980CC8883
:10074300F0EF60010E4E60C388F0ED2402B40400A4
:1007530050B9F582EB2402B4040050AF2323458241
:10076300239006C273BB010689828A83E02250026A
:10077300E722BBFE02E32289828A83E49322BB0140
:100783000CE58229F582E5833AF583E0225006E9F8
:100793002582F8E622BBFE06E92582F8E222E582FD
:1007A30029F582E5833AF583E49322BB0106898226
:1007B3008A83F0225002F722BBFE01F322EF8DF071
:1007C300A4A8F0CF8CF0A428CE8DF0A42EFE22BCDA
:1007D300000BBE0029EF8DF084FFADF022E4CCF8CE
:1007E30075F008EF2FFFEE33FEEC33FCEE9DEC9833
:1007F3004005FCEE9DFE0FD5F0E9E4CEFD22EDF8B9
:10080300F5F0EE8420D21CFEADF075F008EF2FFF5B
:10081300ED33FD4007985006D5F0F222C398FD0F43
:10082300D5F0EA22C2D5EC30E709B2D5E4C39DFD89
:10083300E49CFCEE30E715B2D5E4C39FFFE49EFED3
:100843001207D2C3E49DFDE49CFC80031207D2305F
:10085300D507C3E49FFFE49EFE22A3F8E0C5F0257D
:10086300F0F0E582158270021583E0C838F0E822C3
:10087300E88FF0A4CC8BF0A42CFCE98EF0A42CFC24
:100883008AF0EDA42CFCEA8EF0A4CDA8F08BF0A4A2
:100893002DCC3825F0FDE98FF0A42CCD35F0FCEB01
:1008A3008EF0A4FEA9F0EB8FF0A4CFC5F02ECD39C6
:1008B300FEE43CFCEAA42DCE35F0FDE43CFC2275BD
:1008C300F008758200EF2FFFEE33FECD33CDCC332E
:1008D300CCC58233C5829BED9AEC99E58298400C96
:1008E300F582EE9BFEED9AFDEC99FC0FD5F0D6E474
:1008F300CEFBE4CDFAE4CCF9A88222B800C1B9005A
:1009030059BA002DEC8BF084CFCECDFCE5F0CBF9BA
:100913007818EF2FFFEE33FEED33FDEC33FCEB33B2
:10092300FB10D703994004EB99FB0FD8E5E4F9FAE0
:10093300227818EF2FFFEE33FEED33FDEC33FCC9C5
:1009430033C910D7059BE99A4007EC9BFCE99AF958
:100953000FD8E0E4C9FAE4CCFB2275F010EF2FFFC7
:10096300EE33FEED33FDCC33CCC833C810D7079B31
:10097300EC9AE899400AED9BFDEC9AFCE899F80F94
:10098300D5F0DAE4CDFBE4CCFAE4C8F922C3E49F62
:10099300FFE49EFEE49DFDE49CFC22EB9FF5F0EA60
:1009A3009E42F0E99D42F0E89C45F022E8600FEC9E
:1009B300C313FCED13FDEE13FEEF13FFD8F122E694
:1009C300FC08E6FD08E6FE08E6FF22E493FC74015A
:1009D30093FD740293FE740393FF22E6FB08E6F98A
:1009E30008E6FA08E6CBF822E493F8740193F97465
:1009F3000293FA740393FB22ECF608EDF608EEF685
:100A030008EFF622ECF0A3EDF0A3EEF0A3EFF02253
:100A1300A42582F582E5F03583F58322FAE6FB0807
:100A230008E6F925F0F618E6CA3AF622D083D08212
:100A3300F8E4937012740193700DA3A393F87401F7
:100A430093F5828883E4737402936860EFA3A3A38E
:100A530080DFEF4E6012EF60010EEDBB010B898268
:100A63008A83F0A3DFFCDEFA2289F05007F709DF5F
:100A7300FCA9F022BBFEFCF309DFFCA9F022E5434D
:100A8300242FF8E6054322782C303702782FE475BB
:100A9300F001120A1F0207682030EB7F2ED230804C
:100AA30018EF540F2490D43440D4FF30340BEF2488
:100AB300BFB41A0050032461FFE5446002154405E6
:100AC30047E5477002054630370D782CE475F00191
:100AD300120A1FEF0207AE0218F87403D23780031D
:100AE300E4C237F5438B2C8A2D892EE4F544F54671
:100AF300F547E54460077F20120ABC80F57545FF82
:100B0300C231C230C232C233C235C236C238120A0F
:100B13008AFF700D3037057F00120ACDAF47AE460E
:100B230022B4255FC2D5C234120A8AFF24D0B40A84
:100B330000501A75F00A784430D50508B6FF01064F
:100B4300C6A426F620D5047002D23380D924CFB4AC
:100B53001A00EF5004C2E5D234020DBAD23180C676
:100B6300D23080C0D23280BCD2D580BAD23580B4E4
:100B73007F20120ABC2032077401B5440040F112F1
:100B83000A81FF120ABC020AF5D238D236809512C6
:100B93000A81FB120A81FA120A81F94A4B7006791B
:100BA300B17A0E7BFF20322EE544602A7E008E82CE
:100BB30075830012078160060EEE654570F0C2D59D
:100BC300EBC0E0EAC0E0E9C0E0EE120E1AD0E0F9B3
:100BD300D0E0FAD0E0FB120768FF60AAEBC0E0EABE
:100BE300C0E0E9C0E0120ABCD0E02401F9D0E0344F
:100BF30000FAD0E0FBE5450460DCD545D98087D217
:100C03003280A2120DFD60F7E545700104120483E2
:100C1300A945600DE545600914F545120EA4EF6082
:100C2300F3EA30E702F404C3995077EAF425450464
:100C330030E701E404F545800D120DFD60C1EA05BE
:100C4300452545120483EA7842F630E701E4254559
:100C530004D5450420350114120E1AE4C0E0120E27
:100C6300A47842E6601320E70714F6120AA4802250
:100C730004F6D0E014C0E07F00120AA4E545600743
:100C8300120A9B1545800B303503120A9BD0E002F4
:100C93000AF5D0E00480C5120DFD60A0E5450412FD
:100CA30004837842EAF6E545203502600104240412
:100CB300120E1A74FF04C0E0120EA4120AA4E54532
:100CC3002035026003120A9BD0E0B545E87F451248
:100CD3000AAE7842E67F2B30E7047F2DF404C0E0B0
:100CE300120ABCD0E075F00A84C0F0120AA5D0E065
:100CF300120AA5020AF5791080027908C236C238B1
:100D03008008D2D5790A8004790AC2D5E5450470F2
:100D130002F545E4FAFDFEFF120A81FC7B0820314F
:100D230013120A81FD7B1030300A120A81FE120A67
:100D330081FF7B20EC3382D592D55013C3E430304E
:100D4300069FFFE49EFEE42031039DFDE49CFCE44A
:100D5300CBF8C231EC700CCFCECDCCE824F8F870D0
:100D6300F38017C3EF33FFEE33FEED33FDEC33FCBB
:100D7300EB33FB994002FB0FD8E9EB303105F8D098
:100D8300E0C448B231C0E00AEC4D4E4F78207B00FE
:100D930070C2EAB5450040BCC0E0120E1CD0F0D0D2
:100DA300E0203104C4C0E0C4B231C0F0120AA5D0BF
:100DB300F0D5F0EB020AF5120A2F0B92530CF958F7
:100DC3000B634C0B5F420CFD4F0D05440D05490BA6
:100DD30078430D0B550C3C460C9A450C06470ED137
:100DE300500B672D0B6B2E0B8E2B0B6F230B8C2055
:100DF3000EBA2A0B274800000B86E545B4FF03759E
:100E03004506120A81FC120A81FD120A81FE120AAA
:100E130081FF783B0204B2790AA2D520331430351E
:100E230009B910020404B9080104A2D520360250FE
:100E330001042032689232B544005034C0E07F2070
:100E43003033197F30A23272367235500F120E735F
:100E5300C232C236C235C2387F30800F303503E923
:100E6300C0E0120ABC303503D0E0F9D0E0B544CC81
:100E73003035177F30B9100C120ABC7F5830340755
:100E83007F788003B90803120ABC3032057F2D0234
:100E93000ABC7F202038F87F2B2036F32292328041
:100EA300CF7F00B407005005243BF8E6FF22286EED
:100EB300756C6C2900D231120A813031F8C2317855
:100EC3004430D50108F6020B272D50434958120A26
:100ED300812403B405004001E4900ECC93120AADC3
:100EE300743A120AADD233754404020CF90122009C
:100EF30001200001230001210041842F0001910002
:100F030044842500000000418430004184240041D2
:100F1300842E0041842C004184220041820600413A
:100F230081040041810500448318000000004A83C6
:100F330031000000000000000000004A8327000089
:100F43000000000000000000448310000000004285
:100F5300830E000041831500418341004283050055
:100F6300004183160042833F1C2044830700000096
:100F73000041830C0041830D0041830B00448342F5
:100F8300000000004183470041834800418346003D
:100F93004483230000000044833B0000000044839B
:100FA30001000000004283200000418317004183B9
:100FB3002200418314004A83CF0000000000000098
:100FC30000FF004A83D90000000000000000FF007A
:100FD3004283E300004283F300004E83E5000000F8
:100FE30000000000000000000000004183F6004103
:100FF30083F5004A84420000000000000000FF0067
:1010030042844C00004A844E0000000000000000AF
:10101300FF00428458000042845E00004184600067
:101023005683F70000000056000000000000000097
:1010330000000000FF00000000028782070289828F
:10104300074C84151F1C1F1E1F1E1F1F1E1F1E1F44
:1010530041800000028F000001240001250042832B
:10106300C600004283C300004283AF00004283B145
:1010730000004283B300004283B500004283B700FF
:10108300004283B900004283BB00004283BD0000DD
:101093004283AD00004183CD004183CE004183AC48
:1010A300004183A8004183C5004183CC004283A64D
:1010B30000004283BF00004183AB00003A70FA8313
:1010C300BCAAE9E43E81E0F8BF9DE9E63F80000069
:1010D30039283C1ABB9969663DA335E3BF255DE713
:1010E3003FC90FDB418DDBCCC44936EE45C9913F87
:1010F300C5B0F83D3F800000C317F534452FFA73A0
:10110300C60AFDDD1211AE04A2E192301420E015EF
:101113009010BF74041205B580261211AE30E1029F
:10112300B23020E0EB8C288D298E2A8F2B9010D3A0
:1011330074041205B5A828A929AA2AAB2B1201A069
:10114300ED4C6007303004EC6480FC221211AEC019
:10115300E08C288D298E2A8F2B9010F774031205AB
:10116300B5A828A929AA2AAB2B1201A0ECC528FCF3
:10117300EDC529FDEEC52AFEEFC52BFF9010E774E0
:10118300031205B5D082A828A929AA2AAB2BE58288
:1011930030E0071202A9B23080A6EFCBFFEECAFE01
:1011A300EDC9FDECC8FC1202A98095ED33EC547F28
:1011B300CC33923024605007D0E0D0E002046E7B41
:1011C300837AF97922783E1201A0EDF933ECF833F2
:1011D30024815011EFFBEEFA1204021203C4ECB2A5
:1011E300E7FC1200AFED33EC33602F2403F8C31395
:1011F300FCED92E7FDE82481E4501FECF8EDF9EEF5
:10120300FAEFFB120402EF04C2E0FCF5821203CEF4
:10121300ECB2E7FC1200AFE58203FAED33EC336086
:10122300071413FCED92E7FDEA22257325303262A1
:10123300642E252D303262640056657200444220CC
:10124300454D505459002573252D303262642F25A6
:101253002D303262640044423A00257300446566CF
:1012630061756C740044657461696C7300436F6DE0
:10127300666F727400536E204661696C00536E2072
:10128300476F6F6400523A4C6F6769633000523A9C
:101293004C6F6769633100523A4C6F676963320080
:1012A300523A4C6F6769633300523A4C6F67696314
:1012B3003400523A43697479202000257320253382
:1012C3006275004D41583A00257325336275004914
:1012D3004C4C553A002573252D3375004156473A3A
:1012E30000553A20204B696C6F00553A20204D6918
:1012F3006C65004C414E47203A4742004C414E47F3
:10130300203A4E4C004C414E47203A5350004C413A
:101313004E47203A46520025733A20202532626414
:1013230000474D540025733A202D25326264004254
:10133300454C4C3A4F46460042454C4C3A4F4E20A2
:10134300004E6F20557365720055252D3375204C63
:1013530041543A2530337540202530322E303266E1
:101363002720256320004C4F4E203A25303375400B
:10137300202530322E30326627202563202020207E
:101383002020202000BE1249253E4CCCCDBEAAAA67
:10139300AB3F8000003E7ADBB03EED63383F24BCB8
:1013A3007D3F490FDBED33ECC2E7CC339230B4FF22
:1013B30013ED547F600302046E7FDB7E0F7DC97CD7
:1013C3003F0214A3C231C3947F401E7007EDD2E7DE
:1013D30094904015EFFBEEFAEDF9ECF87F007E00F8
:1013E3007D807C3F1202A9D231ED33EC332484306B
:1013F300E705E4C0E0806D04FAEDD2E754F0C333AF
:10140300DAFD540734002323C0E0CCC0E0F8EDC07C
:10141300E0F9EEC0E0FAEFC0E0FBE41203CEEC2407
:10142300FEFC8C398D3A8E3B8F3C1201A07B007AF7
:10143300007980783F1200AFECC539B2E7FCEDC507
:101443003AFDEEC53BFEEFC53CFFD0E0FBD0E0FA32
:10145300D0E0F9D0E0F81200AFA839A93AAA3BAB23
:101463003C1202A98C398D3A8E3B8F3C90138874C1
:10147300031205B5A839A93AAA3BAB3C1201A0D087
:10148300E0600F2494F582E43413F5831209EB1220
:1014930000AF30310B7BDB7A0F79C978BF1200AF15
:1014A300ED33EC336006ECA23092E7FC22C231C28A
:1014B30032C233C234F9E4F52FF530FCFDFEFFE907
:1014C3001030EA20330CB42D04D233D322B42B02D0
:1014D300D32224D0504794095041240A303415F8BC
:1014E3008530F0740AA42872E74051C5F0704D8529
:1014F300F030D322D232C0E0E4FBFA7920784112F3
:1015030001A0ECF8EDF9EEFAEFFBD0E0FCE41203F6
:10151300CE1200AF3031B4152FD322240A20342049
:10152300B4FE0720311AD231D32224EB600424E025
:10153300700EA2339231D234C233D322C302046E6B
:10154300E430340BE530303302F404A2319233300B
:1015530032EA252F20D2E5A2E792345002F404B4F4
:10156300260050D8CCC0E0EDC0E0EEC0E0EFC0E014
:10157300EC120632D0E0FFD0E0FED0E0FDD0E0FC7C
:101583002034051201A080031202A9303303120391
:10159300B3C32225730052616461724F464600252E
:1015A3007320202533626400566F6C00530053523E
:1015B30000535243005352434800576169742E2E1F
:1015C300002533627500447420253262753A252D57
:1015D30032627500546D20253262753A2532627588
:1015E3000025733A252D332E31665600426174006F
:1015F30025337525400025303262643A2530326246
:10160300643A253032626400257320253362750005
:101613004D41583A005359532043484B004C6F7780
:10162300204261742000257325303262642E252DFB
:1016330030326264005665720053797320476F6FCE
:1016430064002020204F2E4B20200002046E22ED48
:10165300A2E7D2E7F9EC3340F260F3B4FF08ED54AC
:101663007F70E8020478F82481C2E0C0E0F4042823
:10167300FAC313FCED92E7FD8C318D328E338F3438
:10168300EEA2E7E9BA7F02C31334009400FA75F0BF
:1016930091A4E5F013F494FE8AF0A433E5F0332427
:1016A3008CD313FDE492E7FE7F007C3F758302EC4D
:1016B300C0E0F8EDC0E0F9EEC0E0FAEFC0E0FBAC4B
:1016C30031AD32AE33AF341202A9D0E0FBD0E0FA31
:1016D300D0E0F9D0E0F81200AFED6480FD30E7010F
:1016E3001CD583CBED33CC33F8D0E0A2E71328C36A
:1016F30013CC13FD22758191021739021D68E493FF
:10170300A3F8E493A34003F68001F208DFF48029F1
:10171300E493A3F85407240CC8C333C4540F4420E0
:10172300C8834004F456800146F6DFE4800B0102CF
:10173300040810204080900EF0E47E019360BCA367
:10174300FF543F30E509541FFEE493A360010ECF1D
:1017530054C025E060A840B8E493A3FAE493A3F847
:10176300E493A3C8C582C8CAC583CAF0A3C8C58207
:10177300C8CAC583CADFE9DEE780BE4B203E20200E
:10178300202532626475004B203E3E2020253262C4
:1017930064004B203E3E3E2025326264004B613E96
:1017A30020202025326264004B613E3E20202532FA
:1017B3006264004B613E3E3E2025326264004B75FD
:1017C3003E20202025326264004B753E3E202025BA
:1017D300326264004B753E3E3E2025326264002037
:1017E30050554C534520200003060912191C242789
:1017F3003038448F348E338D328C31AB38AA37A9CD
:1018030036A8351202A91213A88F348E338D328C69
:1018130031E53530E747ECC0E0EDC0E0EEC0E0EF86
:10182300C0E0E4FFFEFDFCAB34AA33A932A83112B9
:1018330003467BDB600250087A0F794978408006C3
:101843007A0F794978C0D0E0FFD0E0FED0E0FDD038
:10185300E0FC1200AF8F348E338D328C31AF34AE57
:1018630033AD32AC31228B288A29892AAB2BAA2C9F
:10187300A92D120768FEAB28AA29A92A120768FF17
:101883006E702BEF600DE52F152F7002152E14458A
:101893002E70037F00227401252AF52AE43529F5E9
:1018A300297401252DF52DE4352CF52C80BEAB28AC
:1018B300AA29A92A120768FFD3EE6480F8EF64808F
:1018C3009840037F01227FFF222020202020202018
:1018D300200025346C752000253362750025372ED2
:1018E30031660020253262642025303262640001B3
:1018F30006080C0E0FEFB40A07740D121903740ACD
:10190300309811A899B8130CC2983098FDA899C2C1
:1019130098B811F63099FDC299F5992225733A25A5
:101923003375004144440044454C202020202000CE
:1019330044454C00454D50545920202000EFC3949A
:10194300094005EF940E4003BF2003D38001C32257
:101953004A414E4645424D41524150524D41594AEA
:10196300554E4A554C4155475345504F43544E4F9E
:101973005644454353415453554E4D4F4E5455458C
:1019830057454454485546524900000000000000A2
:101993004F4F000006000600287F147F0A242A7F89
:1019A3002A12221008042236495522500000000B47
:1019B30007001C2241000041221C003E7F7F7F3E26
:1019C30008083E08080000005838080808080800FE
:1019D3000040000020100804023E5149453E0042E9
:1019E3007F40004261514946224149493618141249
:1019F3007F1027454545393C4A494930017109055E
:101A0300033649494936064949291E00363600003E
:101A1300005B3B000000081C3E7F14141414147F69
:101A23003E1C0800020159090600060600007E114B
:101A330011117E417F4949363E41414122417F4157
:101A4300413E7F494941417F090909013E414949D5
:101A53007A7F0808087F00417F41002040413F0111
:101A63007F081422417F404040407F020C027F7F69
:101A73000204087F3E4141413E7F090909063E4178
:101A830051215E7F09192946264949493201017FBF
:101A930001013F4040403F07186018073F4038406E
:101AA3003F631408146307087008076151494543ED
:101AB300007F41410002040810200041417F0004DF
:101AC300020102044040404040000402010020544F
:101AD3005454787F48444438384444442038444478
:101AE300487F3854545408087E090200081454549B
:101AF3003C7F0804047800447D40002040443D00BE
:101B0300007F10284400417F400078041804787C4B
:101B13000804047838444444387C142424181824D2
:101B2300147C40007C0804044854545420043E446C
:101B330020003C4040207C1C2040201C3C40304086
:101B43003C44281028444C5050503C4464544C446A
:101B53000008364100000077000000413608000805
:101B6300040810082A552A552A6060606060707066
:101B73007070707C7C7C7C7C7F7F7F7F7F007F3E6E
:101B83001C08007F22140800060600006F12651966
:101B9300602927202F624F49794949601F60007FE0
:101BA3002A292D296A41413F087F79494F007F0047
:101BB30000040404040810207F0000007D00446436
:101BC300544C4438444444387C0404040C094949C3
:101BD300291F7F08000000007F41417F087F007FAD
:101BE30000794949494F7F0800000020100F102059
:101BF3007F08000000414171415F111171111769A4
:101C030049474F420000000000094949291F087F46
:101C13000000005F5454545F6649494F02000000BE
:101C23000000004141211F7F087F00004669496988
:101C33004675555557754C4271424C004141211F21
:101C4300087F007F00003E41413E7F000000005FAF
:101C530055555555417141715F42221F22427F08FC
:101C630000000012011001000000088304000000BE
:101C7300010102000109092100010001222E0009CE
:101C8300022200010100C0FA090400000103000060
:101C930000092100010001222E000705810308002D
:101CA3006400002E06A0FF09A5A10109A609A51538
:101CB30080257F75089540B10209A71580257F759A
:101CC300089508810209A91580257F75089540911B
:101CD30002C0040309041A03570049004C004C00D6
:101CE3002000540052004E004900430053000000FE
:101CF3001803470050005300200041004C004500EA
:101D03005200540045005200FF1CD5FF1CD9FF1C94
:101D1300F3000000000000000000000000000000CD
:101D23000099A3ADB8C2CCD6E0EBF5D14912281087
:101D3300122792C29312293B122CE8124875124DB6
:101D4300B8124FFB12315A125CC7124192E4F522CA
:101D5300F523F521F5259083F6F0D20C90842CF031
:101D6300F1FA020006B12E7F407E0D7D037C001246
:101D73002C4D122D0AE47F107E27FDFC122C4D12F0
:101D8300412A30260CD293D227122FE4125D6980A8
:101D930004C293C227125C521238FEEF640A7053D6
:101DA3001239A8EF603D24FA704912243A122A2608
:101DB3009083E3E07002A3E0700312294D900013B7
:101DC300E054FDF0A20DB3920D9083E3E07002A303
:101DD300E060089083D8E0FF122BE0201915122C45
:101DE300958010900013E06402F01250D11251025A
:101DF30012488EF1FA30271E202A1B201A18201BA6
:101E030015201C12201D0F201E0C201F09125A82A0
:101E1300BF0103122DBB300823202A2020291D20B7
:101E23001A1A201B17201C14201D11201E0E201F00
:101E33000B12293B90842AE0FF124434122CE8123F
:101E430028A8F1BEA198902000E0F52030003DE4E1
:101E5300908423F09084317408F090842D7405F0FD
:101E6300E4908429F090842AF090842B740DF0C2BE
:101E730001C202C200125DCFE4F524D226FD7C200C
:101E83007F011222EB124FDDD1DCF1CC902000E078
:101E9300F520A3E0908423F0902002E0908431F0B9
:101EA300902003E090842DF0902004E090842AF0A9
:101EB300902005E0908429F0902006E090842BF098
:101EC300902007E0F524781C7C837D017B017A60F8
:101ED30079007E007F040207421222EBAB207D00D3
:101EE3007C207F01F13F908423E0FB7D017C207FF8
:101EF30001F13F908431E0FB7D027C207F01F13FC3
:101F030090842DE0FB7D037C207F01F13F90842AA8
:101F1300E0FB7D047C207F01F13F908429E0FB7D81
:101F2300057C207F01F13F90842BE0FB7D067C2024
:101F33007F01F13FAB247D077C207F018C2C8D2D0D
:101F4300E4FEF9BF010812242D902555801CBF0221
:101F5300081224209045558011BF030812241390C2
:101F6300655580061222DE90855574A0F0F1F3EBDF
:101F7300F0530380F1F3125E90B503047E018005F4
:101F8300BC20027901EE7003EC60E9E9640170287A
:101F9300F1F3E05480B503027E01BF01059025559E
:101FA3008013BF0205904555800BBF03059065550F
:101FB300800390855574F0F0AF062230090A7D0046
:101FC3007C207F01D1DCC20922E4FBFD7C607F031E
:101FD300F13FE4FB7D017C607F03F13FE4FB7D0285
:101FE3007C607F03F13FE4FB7D037C607F03E13F83
:101FF300852D82852C8322300C3390842CE025E0C0
:1020030025E04422F597E59730E0FB90842CE0FF30
:102013007006908422E596F0EFC3940050089084F4
:102023002CE004F08005E490842CF0C20C22E490B0
:102033000005F0900003F090000774FFF0E49000B7
:1020430009F09000137407F09000157402F09000EB
:102053001714F09000B07438F09000B47430F0901E
:1020630000C77401F0228C528D53E4FEF9BF0107BF
:10207300912D9025558019BF0207912090455580D9
:102083000FBF03079113906555800551DE90855569
:1020930074A0F011E4EBF053038011E4125E90B5E9
:1020A30003047E018005BC20027901EE7003EC601D
:1020B300E9E96401702811E4E05480B503027E016C
:1020C300BF01059025558013BF0205904555800B30
:1020D300BF0305906555800390855574F0F0AF06F6
:1020E30022855382855283228F488B4B8A4C894D9C
:1020F300CEECCECFEDCF8E508F51E54F154FAE4E78
:102103007002154E4E602E1258547002054C14F98D
:10211300120768FBAD51AC50AF4811690551E55149
:10212300AE507002055014F5828E83E0FF90804616
:10213300E02FF080C522908083E0600221C9908067
:1021430001E024FD600221C9908082E0FE7032EF3D
:10215300D394014071EF24FFFDE434FFFC9080052C
:10216300E0FAA3E0FBC39DEA9C5008CCEACCCDEB9C
:10217300CD8004EF24FFFD7881EDF6EE0408F680B0
:102183001BEFFDC3908006E09D31CA5005A3E0FF1D
:1021930080007881EFF6908082E008F6908002124A
:1021A30058EB7882E62483F9E43480FA7B0118E65D
:1021B300754E00F54F11EB788151947009908001B1
:1021C300F0A3E0FF51B722908005E09400228F48EE
:1021D300908081E06037E5486002419390804174CC
:1021E30005F0908001E0908042F09000E0E0908064
:1021F30043F09000E2E0908044F078C47C807D015D
:102203007B017A8079417E007F4002074290800102
:10221300E024FC705DE5487020C3908006E09407DD
:1022230031CA5005A3E0FF80027F077881EFF6757E
:102233004801E49080C4F08016C3908006E09408BF
:1022430031CA5005A3E0FF80027F087881EFF69042
:102253008003E0FEA3E0FF74C42548125A25788169
:10226300E6754E00F54F1258235194702390800168
:10227300F022E47882F67882E6FFC394085011E5F1
:10228300482F24C4F582E43480F583E4F00680E625
:1022930022E6FF7E00908004E02FF0908003E03E72
:1022A300F0C3908006E09FFF908005E09EFEF0A3C0
:1022B300EFF04E22BF0107912D9025558019BF02E3
:1022C300079120904555800FBF03079113906555E3
:1022D300800551DE90855574F0F02290855574AADF
:1022E300F0908AAA7455F0228C2C8D2DE4FEFDBF4C
:1022F3000109912D7177902AAA8028BF020C9120A1
:10230300904555717A904AAA8019BF030C91139096
:102313006555717A906AAA800A51DE908555717A63
:10232300908AAA7455F0121FF37430F0121FF3123F
:102333005E86BB80047E018005BA20027D01EE70BB
:1023430003EA60E8ED64017028AB04530380BB80AB
:10235300027E01BF01059025558013BF02059045FC
:1023630055800BBF0305906555800390855574F028
:10237300F0AF06229025557480F074AAF0228C48A1
:102383008D49E4FEFDBF0109912D7177902AAA8042
:1023930028BF020C9120904555717A904AAA801962
:1023A300BF030C9113906555717A906AAA800A5104
:1023B300DE908555717A908AAA7455F08549828595
:1023C30048837430F0854982854883125E86BB80DA
:1023D300047E018005BA20027D01EE7003EA60E508
:1023E300ED64017028AB04530380BB80027E01BF00
:1023F30001059025558013BF0205904555800BBFFD
:102403000305906555800390855574F0F0AF06225F
:1024130090655574AAF0906AAA7455F022904555B8
:1024230074AAF0904AAA7455F02290255574AAF024
:10243300902AAA7455F022125DC71209FB200802E4
:1024430081EE90844EB107125D7AB1079083351205
:102453000A07908406E07002A3E060407E837F3128
:102463007C837D27124396125D8D7FE87E03FDFCFE
:102473007854125E3650028006125DC71209FB9033
:10248300831CB107124346125DD4908318B107121F
:102493004346908318120A07D20F8034C20FA20F4B
:1024A300300E01B3502A124FDD51EB90831CE0FB39
:1024B3007D00121FED90831DE0FB7D01121FED9047
:1024C300831EE0FB7D02121FED90831FE0121FEAC3
:1024D30090844EB107908327125D7DB10790832BC3
:1024E300120A07300F03D20E22C20E227855E6FEDF
:1024F30008E690E00475F00A120A13EE75F00AA4D8
:102503002583F583E0FCA3E0FDA3E0FEA3E0FF2227
:10251300122935C1EE301102C1F3301002C1F3901C
:102523008458E07002A3E07011752FFF75301375A6
:102533003144122DB2122CE8C1A3125D1F91F8E4AD
:10254300FB12001D785560025007125D2191F8803F
:1025530008125D2191F81203B3125D32125DDA1293
:102563005D1F91F8E4FB12001D9084616002500F1F
:10257300125CDDC00412438F125D1F91F8801912A3
:102583005CDDC004C005C006C007125D1F91F812D0
:1025930003B3D003D002D001D0001200AB125D17F9
:1025A300125E69752FFF75301375314C7855E6FA55
:1025B30008E6FB2401F533E43AF5329084611247CF
:1025C3007E124426F5398E388D378C3690E0001212
:1025D3005E0591FFE4FB12001D7F53600250027FF2
:1025E3004E8F3A7B017A837949120ADD7857A60622
:1025F30008A60791EFE4FB12001D78556002500412
:1026030091F1800591F11203B3125D32125DDA91FB
:10261300EFE4FB12001D9084616002500C125CDD3C
:10262300C00412438F91EF8016125CDDC004C00515
:10263300C006C00791EF1203B3D003D002D001D07C
:10264300001200AB125D17125E697857E6FE08E6CA
:102653002449F974833EFA7B01C003C002C00175AB
:102663002FFF753013753169908461E0F532A3E073
:10267300F533124426F5378E368D358C3491EFE4DD
:102683001B12001D7F57600250027F458F38D00117
:10269300D002D003120ADD7B017A8379491241FA11
:1026A30030141AD37856E6940018E69400400708CD
:1026B300E61618700116C214200230802730132B3F
:1026C300908459E024FFFF908458E034FFFEC378E0
:1026D30056E69F18E69E50070806E618700106C2E4
:1026E30013200207E4FD7F13122B8B122CE8A11891
:1026F30022301702E19112293BD2179083F712443B
:1027030029125D94B107123D1C90844EB107125DEE
:102713007AB107908335120A0790844EB1079083EC
:1027230027125D7DB10790832B120A0712479790FA
:1027330083F7B107908307125D4A9083F7B10712BD
:1027430008FE90830CEF123D149083F7B107123EFD
:10275300ADAF0590830D123D139083F7B1071208B7
:10276300FE90830BEBF01247771247B2E4FB12485B
:1027730042122CE81236CE12293BE4908406F0A3D1
:10278300F07F807E847D1EFC122C4D12293B22C2D9
:10279300AFD2A8C2B8C289D288D2AAC2BAC28BD2D7
:1027A3008A5389F0438902758CA1E4F58AD2B9D2A0
:1027B3008CD2A9F5C8D2BD75CD6375CB6375CCC07A
:1027C30075CAC0D2ADD2CAC299C28E43878053891B
:1027D3000F438920758DECD28E908104F090810592
:1027E300F0759850C299C298D2ACD2BC439101758E
:1027F300950343972075940875B10875B20775B3AF
:102803000875B40775A13143A710D2AF2290843164
:10281300114812410512000E1257A975E10275EA1B
:102823003875EA1875EC0C75EB2875E6BA75E6BED3
:1028330075EB2275E9BF75EE80F5E875B70143A71F
:102843000122F0D209E0901D2393F5A22220105417
:10285300908305E07002A3E0604A30131390843143
:10286300E0C3940A5004E0041145F1D6C213801466
:10287300301411908431E0D394004004E0141145E6
:10288300F1D6C214752FFF7530157531A27532FF5D
:102893007533157534AB908431E075F00AA4B1B08B
:1028A30091E880A922300818A210B0155012908424
:1028B30008E0F46009E4FD7F13718B124F1BC21013
:1028C300A21682125008F156C216C2128061A215D6
:1028D3008212502E313BC212C215D209C227C293B3
:1028E300C226752FFF7530157531967532FF753316
:1028F30015753499B1B212315A125CC791E8D1DD22
:10290300802DA211B0155017120006313B2002068C
:10291300E4FD7F13718B124C4F313B91E88010A281
:10292300147213500AC213C214313B1150313B02CB
:102933000006E47855F608F6752FFF7530187531E3
:10294300CC7B017A837971020ADD125DC71209FB20
:10295300313B90844CE07002A3E0700C1234F5908C
:10296300844CEEF0A3EFF022201B277A847B427D78
:10297300167FBC7E0251106012E45119600DD21B08
:10298300D1D7908429E0FD7F098025E45119704B4C
:102993008046201C2A7A847B427D167F2C7E01513F
:1029A300106015E451196010D21CD1D7E4FD7F17D4
:1029B300718BF1E4914D8023E45119701E8019202D
:1029C3001A197A847B42510A6009E451196004D2CE
:1029D3001A8008E45119700312510290844CE0707C
:1029E30002A3E060157A847B42125D84511960076B
:1029F300E47FFF511A7003125102301B09123EC0CB
:102A03009083717455F0227D5A7F0F7E00710A788E
:102A1300541209FB74FFFFFEFDFC78541209DEC358
:102A230002099E125DC71209FB9083F5E0FFA3E044
:102A330004F0C39F4002E4F0124D5CFF9083F6E084
:102A4300FE044F9000E0F0D2AFEE25E024E5F582DE
:102A5300E43483F583E0FFA3E09083F3CFF0A3EFA7
:102A6300F0313B1231F8EF4E602F7E837FCF7C84B1
:102A73007D4E12439678541209FBD21DC21EC21F0B
:102A8300200202F1D6D1DD12512B9083D8E0FF1240
:102A9300517EF1E4914D123EC09083E3E07002A3B6
:102AA300E06063301D60201E297A837BCF7D167F13
:102AB3002C7E0151106014E45119600FD21E123E96
:102AC300C09083D8E0FF1247158023E45119701E8C
:102AD3008019201F197A837BCF510A6009E45119A9
:102AE3006004D21F8008E4511970031250D17A8315
:102AF3007BCF125D8451196004511770031250D1BA
:102B030012512B123EC0228E288F298D2A8A2B8B9D
:102B13002CE4FFFEFDFC125E1C124396125E1C1297
:102B230036D97871A607E6FFF46053908456E0FB2C
:102B3300AD2A123457EF6043125E7CF583125E7246
:102B430050091234EEED24B4FB800A125E7C123479
:102B5300E8AF05AB077871E6FFAD2A123457EF6093
:102B630017AE28AF29E4FCFD786D125E3650057868
:102B73006D0209C274FF8007E48004E48001E4FF6E
:102B8300FEFDFC22E4FD7F15ED14600C14600E14B1
:102B93006010240370148012EF24218008EF244274
:102BA3008003EF2463785BF68004785BA607D2B4D6
:102BB300D2B500000000C2B4125466BF01127F01F7
:102BC300F120E4FFF120E4FFF120785BE6FFF12040
:102BD300C2B4D2B500000000D2B47F0122E478541D
:102BE300125C4A908406E0FCA3E018A60408F6EF02
:102BF300C4540F125D3A6031125E0E402820192B27
:102C0300D3EF942CEE94015018B19991E89131E4EB
:102C1300FD7F14718B9145B19B91439131D2198002
:102C23000AC2188006C2198002C2197F0122E4FD7C
:102C33007F14718B7F207EA17D077C00914D313BFA
:102C430091E87F207EA17D077C008F2E8E2D8D2C19
:102C53008C2BE47F207E4EFDFCAB2EAA2DA92CA845
:102C63002BC312099E402AE47B207A4EF9F8AF2E3B
:102C7300AE2DAD2CAC2B1208FE908425120A0790C2
:102C83008425122507EC4D4E4F6006908000E060CE
:102C9300EE22E47854125C4A908406E0FEA3E01826
:102CA300A60608F690842BE0125D3A6033125E0E9E
:102CB300402A20182DD3EF944AEE9401501AB1996B
:102CC30091E871879145E4FD7F15913571879145B1
:102CD300B1999143D218800AC2188006C2188002A3
:102CE300C2187F0122C2C4C2C6E4785BF6785BE6F1
:102CF300FFC39408500C124187E01241AF785B0682
:102D030080EBD2C6C2C522313B309065752FFF756B
:102D13003016753118B1B291E8D1DD125D55E4FB7F
:102D2300FA79207841120346400F752FFF7530164C
:102D3300753120B1B291E8D1DD20021D71877FE0AA
:102D43007E677D357C00914D908429E0FD7F0C7179
:102D53008B7FC07EC67D2D80067F807E847D1E7C1A
:102D630000914DF1E4914DD1E77F407E427D0F808C
:102D73001F752FFF7530167531297532FF753316A0
:102D8300753438125DB6B1B291E87FE07E937D046D
:102D93007C00914D213B313B752FFF75301675310A
:102DA3000B7532FF7533167534137855E6F5357B9D
:102DB300017A837971020ADDE47854F608F6125A2F
:102DC300AF7854A6077F00202A027F017854E67E5D
:102DD3000060027E01EE5F7002C1D6125B8F7855F0
:102DE300A607202E0818E69083C5F0D22E9083C53F
:102DF300E07854666002E0F67854E624FD604314FC
:102E0300607A24026002C1B9F1ED500D752FFF7590
:102E1300301775317E8F32801FF1DC500D752FFF17
:102E230075301775318A8F32800E752FFF75301705
:102E33007531957855E6F532B1B291E8E4FD7F1E20
:102E4300C1CAF1ED500D752FFF7530177531A08F85
:102E530032801FF1DC500D752FFF7530177531ABC4
:102E63008F32800E752FFF7530177531B67855E6A2
:102E7300F532B1B291E8E4FD7F1F804BF1ED500DC7
:102E8300752FFF7530177531C18F32801FF1DC50FC
:102E93000D752FFF7530177531CC8F32800E752F5E
:102EA300FF7530177531D77855E6F532B1B291E831
:102EB300E4FD7F1D8011752FFF7530177531E2B169
:102EC300B291E8E4FD7F30718B7FE07E937D047CDB
:102ED30000914D22E4FD7F17718B7F807E847D1EE0
:102EE3007C00814D313B752FFF75301675313CB138
:102EF300B291E8200216908429E0FD64026002800A
:102F030005908429E0FD7F0F718B8000D1DD313B7B
:102F1300752FFF753016753145B1B281E88F2A12CE
:102F23005466EF64017023785CF6E52A30E704D237
:102F3300B48002C2B40000D2B5E52A25E0F52A0028
:102F430000C2B5785C06E6B408E0125466BF01021D
:102F5300C2B42220117C201079908305E07002A373
:102F6300E0606F30132390842DE0C3940F5007E08B
:102F730004F0D209800690842D7402F0200206E446
:102F8300FD7F13718BC213802430142190842DE0B4
:102F9300D394024007E014F0D209800690842D7484
:102FA3000FF0C214200206E4FD7F13718B12412A35
:102FB300313B752FFF7530127531CB7532FF753389
:102FC300127534D290842DE075F00AA4B1B091E863
:102FD300808122E4FD7F17618B7855E6FFD394054A
:102FE300227F407E427D0F7C0022D2297855E6FF66
:102FF300D3940222C0E0C083C082C0D075D000C089
:1030030007C2A89083CDE004F0E024FE602D146095
:10301300451460562403706B11939083AFCFF0A3D4
:10302300EFF09083AFE0FFA3E09083A9CFF0A3EF8D
:10303300F030B2FD11939083B1804111939083B32B
:10304300CFF0A3EFF030B2FD11939083B5CFF0A38F
:10305300EFF0D228802D11939083B7CFF0A3EFF038
:1030630030B2FD11939083B9801211939083BBCF3B
:10307300F0A3EFF030B2FD11939083BDCFF0A3EF37
:10308300F0C228D2A8D007D0D0D082D083D0E032EB
:103093009083C6E0FFA3E022C0E0C0F0C083C082FB
:1030A300C0D075D008C28C9083C7E004F07006903E
:1030B30083C6E004F09083A7E004F070069083A633
:1030C300E004F030251E30271BC39083C7E094C86B
:1030D3009083C6E09400400C3115315AC295C22545
:1030E300D224C22830241E30271B9083AD31B390E5
:1030F30083C7E09F9083C6E09E400AD225D295C243
:1031030024E4F0A3F0D28CD0D0D082D083D0F0D0FE
:10311300E0322028069083CCE004F09083CCE0D307
:1031230094024002E4F09083CCE014600F14601723
:103133002402701A31527480F0C296229083AD74C7
:1031430005F0A3743C8004315274A8F0D296229007
:1031530083AD7402F0A3229083ACE07018C229C23D
:103163002E9083CEF09083C1F0A3F09083C5F090AE
:1031730083CAF0A3F0C228E49083CDF0125D73906C
:1031830083AFF0A3F09083B1F0A3F09083B3F0A3E7
:10319300F09083B5F0A3F09083B7F0A3F09083B9D8
:1031A300F0A3F09083BBF0A3F09083BDF0A3F022D3
:1031B300E0FEA3E0FFC322E47859F608F6302820A6
:1031C3009083B131B39083B4E09FF69083B3E09ED4
:1031D30018F6E6FF08E69083C1CFF0A3EFF0800D69
:1031E3009083C1E0FEA3E07859A60608F67859E675
:1031F300FE08E6FF22F1F31250B708A60608A60759
:10320300E4125C49F1BE08F1BB786512441D78698C
:103213001209FB12501B785DEEF608EFF6D39414F7
:10322300EE94005004F1F3800A785EE624EC795AB8
:103233001250C01250B724ECFDEE34FFFC785DE66B
:10324300FA08E6FBC39DEA9C4009785BA60608A63C
:1032530007800AEB2414785CF6E43A18F69083F3BB
:10326300E07002A3E07002813CEB4A7002813C787B
:103273005BEAF608EBF67859A60208F6D3785AE625
:10328300940118E69400402B7F1C7E347DCF7CC1D3
:10329300D10E1200AF7859E6FA08E6F1AB120A1321
:1032A300EA9150F1D3600C400A785AE6161870017F
:1032B3001680C9785BF1B49083F4E09F9083F3E0C8
:1032C3009E40297F1C7E347DCF7C41D10E1200AFFE
:1032D300785BE6FA08E6F1AB120A13EA9150F1D3F0
:1032E300500A785C06E61870010680C7F1E34E6069
:1032F30008785AE616187001169083F3E06E70038F
:10330300A3E06F6008785C06E61870010631F07878
:103313005DA60608A607785DF1B4785C96EE18966C
:103323005070F1ABEF914C125E5FF1A29083E1E03C
:10333300B4EE03125ED8125EE1124396786112096D
:10334300FB125EE1D1D97858A607E6FFF46039F1A4
:103353009760359083E1125E72500891EEED24B4CC
:10336300FB80099083E191EAAF05AB077858E6FF4C
:10337300F19C6014F1EB122A1F400DF1EB1209FBD3
:10338300F1E308A60608A607785E06E618700106AC
:1033930080847860E618467002813CE47F207E03D7
:1033A300FDFC7865125E364002813C785FE6FE08DC
:1033B300E69080089149125E5FF1A29083E1E0B448
:1033C300EE03125ED87A837BD97D0F7F587E02127B
:1033D3002B0A7869F1BB7869122A1F605CE4FFFE4F
:1033E300FDFC7869122A1F60509083F6E0FFE4FC2D
:1033F300FDFE7BCC7A0CF9F8120873EF786026FF98
:10340300EE1836FE785DF608EFF69083E3E06E7013
:1034130003A3E06F6023785DE6FF08E69083E3CFC4
:10342300F0A3EFF07A8379D97B0178CF7C83F1A283
:103433009083E3E0FEA3E0FF22E4FEFF227858E658
:10344300FE08E690E00075F00A120A13EE75F00A22
:10345300A42583228F2DAA05125E3DC36480948028
:10346300500891EEED24B4FF8007125E3D91EEAF5C
:10347300057872A607EA252DFFE433FEC364809422
:1034830080500891EEED24B4FF800BE52D2AFFE474
:1034930033FE91EEAF057873EFF618E6FEB507033A
:1034A3007F01227873E6FFEED39F401B18E6D39B80
:1034B3005006EBC394B44009E4D39B5007EB9F50F1
:1034C300037F01227F00227872E6D39B500A08E62D
:1034D300FFEB9F50037F01227F0022120A13EE7538
:1034E300F00AA42583F583E0FF7E007C007DB4020F
:1034F3000827908458E07002A3E07002A1F8E478F2
:1035030058F608F67858F1B4125E495002A1F890C3
:10351300E00075F00AEF1224FB7B1C7A3479CF7834
:10352300C11200AFD10E1203465002A1EE78581219
:103533005D211224F87B1C7A3479CF78411200AFD5
:10354300D10E12034660044002A1EE78581224F112
:103553007B927AB1790978C2F1C5D1111203465031
:1035630002A1EE78581224F17B927AB1790978425C
:10357300F1C5D111120346600250709140AF82FE33
:103583007C847D4ED1D9785AA607E6FFF4605CF1BE
:103593009760587858E6FE08E6FF90E0089149F5F1
:1035A30083E0C374809480501190E00875F00AEFB3
:1035B30091DEAF05ED24B4FB80127858E6FE08E6F1
:1035C30090E00875F00A91DEAF05AB07785AE6FF85
:1035D300F19C60179140FAA9827B0178427C84F1C7
:1035E300A2E490844BF078590250C8785906E61843
:1035F300700106A107125102E4FEFF22120A13EE24
:1036030075F00AA42583F5831209CE90844EE0F861
:10361300A3E0F9A3E0FAA3E0FB2212293B9084582C
:10362300E0FAA3E0FBC39433EA94034002C1BC90E5
:10363300844E12250790E000125E059150F5831227
:103643005D7D12250790E004125E059150F583120B
:103653000A07908456E0C374809480500A91EAAFBD
:1036630005ED24B4FF800790845691EAAF0590845A
:1036730058E0FCA3E0FD90E00875F00A120A13EC91
:103683009150F583EFF090E009125ECF9150F583EE
:10369300E4F0908459E004F07006908458E004F05C
:1036A300908458124F07753319753426125E5412DD
:1036B3002DB2125EB57F0A800F752FFF7530197515
:1036C300312A122DB2124FEB122B8B7F407E4B7D92
:1036D3004C7C00022C4D1247BB853082852F83D151
:1036E300118F828E831225071200AB78721247EF77
:1036F300D1111247C41225051200AB78761209FBCB
:1037030078761209C21247A078721209C21217F60C
:10371300125EFA1201A0125EC61202A912438DE4D0
:10372300FFFE7DE17C431200AB120402787AEEF6D1
:1037330008EFF6F1CC500E18125E2AED2468FFEC68
:103743003401FE800C787A125E2AECC313FEED136B
:10375300FF787AA60608A607E4FFFEFDFC7876123A
:1037630009DE1203467011FFFEFDFC78721209DEBA
:1037730012034670037FFF22F1DBF1CC7D00500280
:103783007D01ED600891EEED24B4FF8006F1DB913D
:10379300EEAF0522908456E0FB7D169157EF227D14
:1037A300017E007F0A02074290800875F00A2278A2
:1037B30054E6FE08E6FFD3221209FB74FFFFFEFD69
:1037C300FC221200AF90845222C3EE6480948022C4
:1037D300F5831209EB020346787AE6FE08E6FF2238
:1037E300785DE6FE08E6FF2278611209C278652259
:1037F3007859760008760122C0E0C0F0C083C08209
:10380300C0D075D000C000C001C002C003C004C056
:1038130005C006C007C2AAC39083A7E0941490838F
:10382300A6E09400403ED3A3E094189083A6E094CE
:103833000150311231B39083C0E09FFF9083BFE00A
:103843009EFE12007ED3EF9404EE648094805014A5
:103853009083ABE004F0E0C3940540089083A87420
:10386300FAF0D22A9083A6E0FFA3E09083BFCFF0C3
:10387300A3EFF09083A6E4F0A3F0D2AAD007D0067A
:10388300D005D004D003D002D001D000D0D0D08254
:10389300D083D0F0D0E032C0E0C083C082C0D07506
:1038A300D01030981EC298908104E02401FFE433C5
:1038B300FE908105E06F7001EE600890810411CFE6
:1038C300E599F0D0D0D082D083D0E032E0FF04F08D
:1038D30074062FF582E43481F58322908105E0FF9D
:1038E300908104E0C39F70037FFF22C2AF908105E4
:1038F30011CFE07855F6D2AFE6FF2211DE7854EF10
:10390300F6F4600FE6FF600B908206E0FE04F031F0
:1039130038EFF07854E6FFF46006EF6003B40ADB97
:10392300908206E0600C2406F582E43482F583E09D
:10393300FF227FFF2274072EF582E43482F583226F
:10394300124FF390837904F0908206E024FBFF90FA
:103953008379E0FEC39F5015A3E0FF3138E0FEEF0B
:103963006E90837AF0908379E004F080DB90837A21
:10397300E0FF12543E908206E02404F582E4348290
:10398300F583E0B5071C90837AE0FF1254509082D0
:1039930006E02403F582E43482F583E0B507037F70
:1039A30001227F0022785476FF752BFF752C00755A
:1039B3002D16752E00752F067B017A827907121852
:1039C30069EF701A3143EF601531EBEF600C7854F7
:1039D30076062017091226F48004E47854F6E4905E
:1039E3008206F07854E6FF22E4FFFEFDFC785512D0
:1039F300441D785912441D785D1209FB7E827F07AE
:103A0300125DF79157125DF7917612040290837954
:103A1300120A079083791225079083F7120A0791F8
:103A2300CA125EEA9083F7122507908342125D4A19
:103A33009083F71225071208FE908347EFF0E0709A
:103A4300037418F0B1159083F7122507D1ADAF05B4
:103A5300908348B1139083F71225071208FE9083D1
:103A630046EBF091CA91F690837D9168B10B91DF9B
:103A7300125DE9C00078551209C2D000125EBE780B
:103A8300591209C2E41203C4125EC61201A0125EE7
:103A9300FA1202A91211077BCE7A6379DE784212F9
:103AA30001A0125D321202A9B10B1201A090831082
:103AB300120A07125DA6C004C005C006C0077855E8
:103AC3001209C2D003D002D001D000125CF212015D
:103AD300A0C004C005C006C007125D291201A0D012
:103AE30003D002D001D0001200AF90837E91E59005
:103AF30083829168B10B91DF125DE9C000785512A2
:103B030009C2D000125EBE125DA6C004C005C00685
:103B1300C00778551209C2D003D002D001D00012D9
:103B23005CF21201A0C004C005C006C007125D29E3
:103B33001201A0D003D002D001D0001200AF9083B5
:103B43008391E59083879168120402AD07AC06E484
:103B53001203C97B187A0979ED91DD125EAC4E60D0
:103B63000BE02402F0908388E03400F091CA125EE7
:103B7300EA30010C908388E0FCA3E091D2125EACA2
:103B830091CA91577889A60608A607908388E070A2
:103B930002A3E0700A908408E090838AF08027787B
:103BA30087E6FE08E6FF788AE624FFFD18E634FF81
:103BB300FC91901247E37C017D681207D2ECC3139A
:103BC300ED1390838AF07889916A12040290838BB3
:103BD300120A07908382E0B4530F90837E12250765
:103BE3001203B390837E120A07908387E0B4570FC2
:103BF3009083831225071203B3908383120A07C2AB
:103C03000890837DE06441704878F77C837D017B75
:103C1300017A837979FE7F161207429083FC12257D
:103C23000790844E120A079084011225079084524C
:103C3300120A07908408E0908456F0E4A3F0D208B7
:103C43009083F7124429125D94122507B11C7F015A
:103C5300227F00220FEFAC0670010E14F5828C83D5
:103C6300E0B42CF022F008E6FE08E6FF7887A6060B
:103C730008A60791577889EEF6FC08EFF6FD7887DA
:103C8300E6FE08E6FFED24FFFDEC34FFFC8E288FF3
:103C9300298C2A8D2B788F7C837D017BFF7A1D797C
:103CA300147E007F0F120742C3E52B9529FFE52AF7
:103CB3009528FEAA28A9297B01788F7C831257981F
:103CC3007A83798F0200367889E6FE08E6FF22FDC3
:103CD300E41203C97BDB7AF9791E783F1201A00253
:103CE3000402120A077889E6FE08E6FF7887A6062B
:103CF30008A60791577889A60608A6077887E6FEDF
:103D030008E6F5828E83E022E4FBFA797A7844228E
:103D1300EDF0E47B64FAF9F822F1F8B1151208FE2C
:103D2300EB24D0FEEA340790840DF0A3CEB114F156
:103D330049D1AD90840FEDF0E47B107A27F147125F
:103D430008FE908410EFF0125D4DD1B71208FE907B
:103D53008412EFB114D1B7D1AD908413B113D1B79D
:103D63001208FE908414EBF0D19554037018FC7D77
:103D7300641207D2ED4C7008D195F1F1ED4C700649
:103D8300908416741DF0908412E0F9FF3395E0FEE1
:103D9300AD30ED3395E0FCEF2DFFEE3CFEC3EF9429
:103DA30018EE648094804027D19EFD908410E00437
:103DB300F0D39D401290840FE004F0A3E0FDD19E68
:103DC300FCED8CF0125EF2908412E0253080291213
:103DD30037CC502A908410E014F094005012908451
:103DE3000FE014F0A3E0FFD19EFEEF8EF0125EF21F
:103DF300908412E02530241875F01884800AE53089
:103E03002975F01884908412E5F0F090840DE0FA9F
:103E1300A3E0FB7C017D6DFFAE021207C0AC06ADD3
:103E230007EBAE027802CEC313CE13D8F92DFBEC09
:103E33003ED194D1B0C3EB9FFBEA9ED194F1F1EF55
:103E43002BFFEE3ACF2494CF34FEFE7C007D071285
:103E530007D2908411EDF07861760190840FE0FF32
:103E63007861E6FEC39F501574142ED1A4FF90848D
:103E730011E02F75F00784E5F0F00680DE908411E1
:103E8300E014FF908410E02F75F00784A3E5F0F0B1
:103E930022FA90840DE0FEA3E0FF2290840FE02439
:103EA30014F582E43484F583E0221208FE7C007D5D
:103EB300640207D2AF2FAE2EAD2DAC2C2278541254
:103EC30009C2F1F8752FFF7530187531D5124839CD
:103ED3007B017A837975120ADDE47F64FEF1545025
:103EE300028012F149B115D312099E500FE47FC825
:103EF300FEF15450079083757484F022F149E47BFA
:103F0300C8FAF9F8D312099E500EE47F2CF15250EF
:103F13000790837474848028F149E47B2C7A01F937
:103F2300F8D312099E5010E47F90F1525009908308
:103F3300737484F0A380099083727484F0A3F0A354
:103F4300F0A3F022F9F8AF2BAE2AAD29AC28227EDC
:103F530001FDFCAB2BAA2AA929A828C302099E8F1D
:103F63002C8E2B8D2A8C29E47854125C4608F60893
:103F7300F6125D4E125E9A1208FE125D417005182C
:103F8300F6087618B115125E9AD1AD7856A60512C9
:103F93005D4D125EA31208FE7857125D437005183B
:103FA300F6087618B115125EA3D1AD7859A605129D
:103FB30037B2785896EE1896400908741826F61802
:103FC300E436F67C007D3C1207C07856E62FFBEC06
:103FD3003EFA08E6FE08E6FF1207C07859E62FFF0F
:103FE300EC3ECFC39BCF9AFE08F608EFF6227C0186
:103FF3007D900207D28F2B8E2A8D298C2822C0E038
:10400300C0F0C083C082C0D075D008C2CF908424D2
:10401300E4F0E5C0F4540333333354F8FFE590F48C
:1040230054074FF0E0FF908430E0FE6F6037EF609D
:104033000E90842EE4F090830504F0A374F4F090C2
:10404300842EE0FFC394645007EE60044222803D57
:10405300EE603AEFC394644034EF94FA502FD215D4
:10406300EE42228028EE60259083057401F0A3744C
:10407300F4F090842EE0FFC394FA5002800CEFB466
:10408300FA0BD216EE422290842EE004F0908424A0
:10409300E0908430F09083A8E06003E014F0908314
:1040A30005E07002A3E0600E908306E024FFF09029
:1040B3008305E034FFF09083ACE06003E014F090FC
:1040C3008421E004F0E0C394324004E4F0D20C9085
:1040D3008425122507EC4D4E4F601C908425A3A325
:1040E300A3E024FFFFEE34FFFEED34FFFDEC34FFCD
:1040F300FC908425120A07D0D0D082D083D0F0D090
:10410300E032D2C6E47854F67854E6FFC3940850FC
:104113000831877420F00680EF122CE87F81314F3D
:1041230090842DE0FF800590842DE0FFE47855F620
:104133007855E6FEC39405500FEE9018F293FEEF08
:104143009E500578550680E8EF4470FF7857A60720
:10415300D2C4C2C6E418F67856E6FFC39408501DCD
:10416300C2C508E6A807FF08800123D8FD30E7048D
:10417300D2C78002C2C7D2C578560680DAD2C6C279
:10418300C5C2C42274712FF582E43483F58322E41B
:104193007854F67854E6FFC39428500F74492FF5EA
:1041A30082E43483F583E4F00680E822FF51448BF4
:1041B3002B8A2C892DE4785CF6E4785DF6785DE64D
:1041C300FFC394085029C2C5AB2B18E6252DF9E48B
:1041D300352CFA120768A807FF08800123D8FD30A1
:1041E300E704D2C78002C2C7D2C5785D0680CE7805
:1041F3005C06E6B405C3228B288A29892AC2C4C275
:10420300C6AB28AA29A92A120768603020112D20DD
:10421300102A201327201424C2C600052AE52A7079
:1042230002052914F912076831AF7F807E1A7D06D3
:104233007C00122C4DD2C6C2C50080C5D2C6C2C5F1
:1042430022EFC394204018EFD394B2501274E02F9E
:1042530075F005A4248CF9741935F0FA7BFF227BE1
:10426300FF7A19798C22752FFF7530187531DB8E23
:10427300328F337B017A837976020ADD12293590F6
:1042830083717441F0A37456F0A37447F0908318BC
:10429300122507EC4D4E4F7002613E90830C717FE7
:1042A30090830D716B90830BE0FFE4FEEB2F714D58
:1042B300908323120A07908347717F908348716B21
:1042C300908346E0FFE4FEEB2F714D908301120AC9
:1042D300079083231236119083019129C39BFFEE2C
:1042E3009AFEED99FDEC98FC90833B120A07E47F5C
:1042F300107E0EFDFC908318123611120873908302
:104303003B1236111208FEE47BE87A03F9F812082F
:10431300FE7855A60608A607300110715818E6FC6A
:1043230008E6123CD28E358F36800B71587855E6ED
:10433300F53508E6F536122DB28005E4FFFE516926
:10434300022CE878541209DEEF2BFFEE3AFEED392A
:10435300FDEC38FC22752FFF7530127531D875329C
:10436300FF7533127534DF22E075F03CA4FFEB2FA9
:10437300FBEA35F0FAED39F9EC38F822E0FF7E007C
:104383007C0E7D101207C0E4FCFDA804A905AA0653
:10439300AB0722F1BBE4FFFEFDFC7872911D78763A
:1043A300911D787A1209FB853082852F831236118D
:1043B300852E82852D831225071200AB7B9A7A19ED
:1043C30079F778411201A07876F1EF123611F1C432
:1043D3001225051200AB9083101236111201A0783A
:1043E3007A1209FB787A1209C2718D1201A0C004F6
:1043F300C005C006C00778761209C2718D1201A0EC
:10440300D003D002D001D0001200AF121652F1E354
:1044130078721209FB78720209C21209FBE4FFFEEB
:10442300FDFC2290845AE0FCA3E0FDA3E0FEA3E0A0
:10443300228F28C3908407E0944A908406E0940175
:10444300400F90830EE0FFA3E0908406CFF0A3EF2C
:10445300F0E528702AB19C9083143001057406F0AE
:104463008003740AF0908314E0D1744002A134F104
:10447300B2300D04E4FB80027B02124842A17CE5CA
:104483002864016002A145908314E0D1744002A125
:1044930032F1A9945A4002E4F09083429129F53015
:1044A3008E2F8D2E8C2D908307122507123F62903D
:1044B3008320EEF0A3EFF0908320E0FAA3E0FB7CEF
:1044C300007D3CFFAE021207D2908317EFF07C0011
:1044D3007D3CAF03AE021207D2908322EDF09083AE
:1044E30041E075F01E8414601614602A24026002F1
:1044F300A17C752FFF7530157531C9D15D8012759B
:104503002FFF7530157531D7908317E0F5329083FF
:1045130022E0F5338060752FFF7530157531E47532
:1045230032FF7533157534EF125D55F1A08047B135
:104533009C752FFF7530157531C4908407E0F532F3
:104543008034908408E0F4601A752FFF7530157578
:1045530031F3E075F002A485F032F533122DB2B1D8
:104563009C8016752FFF7530157531F9D15DE0F517
:104573003390840DF17E122DB2908412E0FF90836C
:1045830016E06F6002F177F197908406E0FFA3E0F5
:1045930090830ECFF0A3EFF022908408E0F4700232
:1045A300C15CE0FF740BD39F500DE0C3942150070F
:1045B300908377744E802E908408E0FF7421D39FFC
:1045C300500DE0C3943850079083777445C15790DA
:1045D3008408E0FF7438D39F5011E0C3944E500B0E
:1045E3009083777453F0A37445F022908408E0FF1E
:1045F300744ED39F500DE0C3946550079083777436
:10460300538051908408E0FF7465D39F500DE0C33D
:10461300947B50079083777453802E908408E0FF37
:10462300747BD39F500DE0C39492500790837774AB
:10463300578021908408E0FF7492D39F5011E0C308
:1046430094A8500B908377744EF0A37457F0229084
:104653008377744EF0A37420F022908410E0F53237
:1046630090840F22EF540FFDEFC4540F75F00AA48A
:10467300FEFFD3908407E09F908406E0940022E439
:104683007859F608F608F6E52454077859F61460C5
:104693001214601E14602A146036146048240570D6
:1046A30068805ED3908407E09414D17B50028059D4
:1046B300804FD3908407E09428D17B5002804A80B6
:1046C30040D3908407E0943CD17B5002803B8031FF
:1046D300F18EFFD3908407E09F908406E095F0501D
:1046E300028026801C9083CDE0D394014019F1CE43
:1046F3009F25E0785BF6E6C3940F5005E418F68037
:104703000C785A760180068000E4785AF6785AE6E7
:10471300FF22D1675003200252ED604F14B408000A
:10472300504990472BF1D87302474302474502474C
:104733004E02475F024752024756024756024763FB
:104743008000908429E0FD7F0E8017F16F8013F1C4
:104753006F800F908429E0FD7F0D8006F16F80024A
:10476300F186122B8B122FE4122C4D22908429E018
:10477300FD7F0F22E4FD7F18022B8BE0F534A3E0CD
:10478300F53522908429E0FD7F042290842BE07587
:10479300F00AA422908412E0908316F0228F388EC0
:1047A300378D368C3522908341E004F0E0C32290AC
:1047B3008412E0FFA3E0FD228E2D8F2E8C2F8D30EF
:1047C30022E52E2404F582E4352D229083B0E0FF08
:1047D3009083B2E02275F003A4C58325F0C583223C
:1047E300E4FBFAF9783F1200AF0204021209FBE579
:1047F300302404F582E4352FF58322123FF830018B
:1048030013112AF9F811237BDB7AF9791E783F1209
:1048130001A08007112A123F4711231139022DB23B
:104823001208FEE40203C4752FFF7530187531E0DA
:10483300E47BE87A03228F358E348D338C32228BDE
:1048430029752FFF7530187531E68F328D337B0153
:104853007A837972120ADDE5297007908375743AB9
:10486300F022E529908375B402047420F022742E9B
:10487300F022E47854F67854E6FFC394FA500B74AC
:10488300072F12393BE4F00680EC2220087612470A
:10489300A994054002E4F012293B908341E0605261
:1048A30024FE601B14602914603724037056752F8F
:1048B300FF7530157531AF7B017A8379728042754C
:1048C3002FFF7530157531B17B017A837973803190
:1048D300752FFF7530157531B47B017A8379748038
:1048E30020752FFF7530157531B87B017A83797583
:1048F300800F752FFF7530157531BD7B017A837974
:1049030074120ADD228F28E47855F6B15C4528F04D
:10491300D2AF7A8079067BFFC001E52875F002A447
:1049230024E3F9748335F0A801FC7D01D001317AC9
:10493300316CE0FEA3E0FFF47002EEF46004EF4E8E
:10494300700B316CE4F0A3F07855F680047855765B
:1049530001316CE0FEA3E0FF9083F4E02FF090833D
:10496300F3E03EF07855E6FF22E52825E024E3F561
:1049730082E43483F583227E007F02020742E478D7
:1049830055125C4612293B9083717453F0A3746EE5
:10499300F0A3743AF030110241D730100241D7909E
:1049A3008305E07002A3E0700241D730131A7859EF
:1049B300E6C39409500506D209800478597601C2EA
:1049C300133002024165801B3014217859E6D394D9
:1049D30000400516D209800478597609C2143002C2
:1049E300024165E4FD7F13122B8B8076301273C274
:1049F30012785A06E6D394044002E4F6785AE62481
:104A0300FE602014602E1460422403705151D8902C
:104A13008374F0EEFF7E007C037DE81207C07856B6
:104A2300EF802051D8908375F0EE75F064A4AEF05A
:104A33007856800F51D8908376F0EE75F00AA4AEC5
:104A4300F0785626F618EE36F6801351D890837711
:104A5300F0A3745FF0EE785626F618E436F6E478A1
:104A630059F6122CE8785AE66404705D12293BB1BA
:104A73005C4401F0D2AF78577C007D007BFF7A80E5
:104A83007902317A7958E7785666700419E718661F
:104A9300601351E3753312753478122DB2C226C2F6
:104AA30027C293801751E3753312753480122DB2E8
:104AB300D226D227D293122FE4125D697FC07EC61D
:104AC3007D2D7C00122C4D21987859E6243090835B
:104AD30078F02198227859E6FE243022C221D2228E
:104AE300752FFF75301275315D7532FF22E47855ED
:104AF300F6E5245407F612293B30110261CB30103E
:104B03000261CB908305E07002A3E0700261CB30B9
:104B130013187855E6C39405500506D2098004E4BA
:104B23007855F6C213200222801930141D7855E6F9
:104B3300D39400400516D209800478557605C21433
:104B4300200207E4FD7F13122B8B7855E614601FB8
:104B530014602F14603F14604C1460552405705E7C
:104B630051E3753312753488122DB2C220800D5172
:104B7300E3753312753491122DB2D220C221C222B1
:104B8300803C51E375331275349A122DB2C220D290
:104B930021C2228029D220D221C22251E3753312AD
:104BA3007534A38016C22051DF7533127534AC807F
:104BB3000AD22051DF7533127534B5122DB2122C7F
:104BC300E87855E6422441FC22E47855F690842A9D
:104BD300E0F6201176201073908305E07002A3E0C5
:104BE30060693014157855E6D39400400516D20950
:104BF300800478557602C21480163013137855E674
:104C0300C39402500506D2098004E47855F6C21312
:104C13007855E690842AF0700A51E375331275349F
:104C230060802090842AE0B4010A51E37533127541
:104C33003468800F90842AE0B4020B51E375331279
:104C4300753470122DB2122CE8808722E47854F662
:104C5300C211301002A15B908305E07002A3E070E3
:104C630002A15B30111F7854E6C3940B500506D2A2
:104C7300098006E47854F6D209C211200207E4FD44
:104C83007F13122B8B7854E670051251EEA15678E0
:104C930054E6B4010471CCA1567854E6B40205126B
:104CA30053F0A1567854E6B403051252AAA15678DC
:104CB30054E6B4040B2026043181A15651F0A156C9
:104CC3007854E6B40504B184A1567854E6B40605D5
:104CD30012427F807E7854E6B4070512525C8073DB
:104CE3007854E6B4080512534B80687854E6B40947
:104CF30005122513805D7854E6640A701A12293B65
:104D0300752FFF75301275312D7532FF753312759E
:104D1300343C125DB68039B15C4402F0D2AF122943
:104D23003BB173BF1F10B165BF0F0B752FFF7530FC
:104D330012753140801A752FFF7530127531497520
:104D430032FF753312753459B1738F35B1658F36B0
:104D5300122DB2122CE8815522C2AF9000E0E0542C
:104D6300F8221209CE78161209AFEF540FFFE4228E
:104D73009080001209CE78111209AFEF541FFFE49F
:104D83002212293B20112D20102A908305E0700266
:104D9300A3E0602090831C1225071247FE30120FF8
:104DA300D209C212125DCFF1DD1222EB121FCC1217
:104DB3002CE880D02278587C847D017B017A40796D
:104DC30000317AD1FE4E6025C3EF9433EE94035045
:104DD30011D14E78007CE07D017B017A407902029B
:104DE3000742E4908458F0A3F0FFFEB1F1228E2A2B
:104DF3008F2B7C407D007F021222EB7C407D009054
:104E03008458D1477C407D01908459D147F1E4AE69
:104E13002AAF2BD14EC37857E69F18E69E50247EC7
:104E230040E6FA08E6FB2402FD74403AFC74002BCA
:104E3300F58274E03AF583D147785706E618700196
:104E43000680CC22E0FB7F02021F3F7C007D0A022A
:104E530007C08E288F2912293BD1FED39400EE94EC
:104E6300005002C1E790844CE0B52808A3E0B529BF
:104E730003125123EF65297003EE65286040E5298D
:104E83006401452860387854A62808A6291237B249
:104E9300125E494029D14E74002FF974E03EFA7B2B
:104EA30001C00174F62FF974DF3EA801FC7D01D027
:104EB300011237A4785506E61870010680CF908456
:104EC30059E024FFF0908458E034FFF0F107753384
:104ED30019753433125E54122DB2125EB57F0B1264
:104EE30036CB8014752FFF753019753137122DB2FB
:104EF300F1EB1236CB7F00227F0122908458E0FE33
:104F0300A3E0FF22E0FEA3E0FFB1F1752FFF7530B0
:104F13001975311F7532FF22908458E07002A3E0A7
:104F23007002E1CEF1F3D1FE908379E0FCA3E0FDC2
:104F3300C39FEC9E4002E1CE90E000125ECF1224AC
:104F4300FF7B1C7A34794F78C01200AF12360E12F1
:104F530003464067F1D590E0001224F87B1C7A34B5
:104F6300794F78401200AF12360E1203466002509A
:104F73004AF1D590E0041224F87B927AB1798978CA
:104F8300C01237C5123611120346402FF1D590E0F7
:104F9300041224F87B927AB1798978401237C512CA
:104FA30036111203466002501290837AE02401FF07
:104FB300908379E03400FED155801390837AE00426
:104FC300F07006908379E004F0E12912361DE4FEC7
:104FD300FF22908379E0FEA3E0227D007C607F03C3
:104FE30022E47856F608F622122CE8E4FD7F12221A
:104FF300E4908379F0A3F022785476017854E6FFA5
:10500300D394075012124908EF60077854E690834F
:10501300F5F078540680E522E4786DF608F611B7CA
:1050230024FF7870F6EE34FF18F6EF4E700201B3EA
:10503300786FE6FE08E6FF786DE6FC08E6FDD39F91
:10504300EC9E5068ED2FFFEC3EC313FEEF13FF7889
:1050530071EEF608EFF608A60608F66D7002EC6E20
:10506300604A7871E6FE08E6FF787066700318E61A
:105073006E60391237ABEF1235FF120346500B78CF
:1050830072E624FF797011C080A67871E6FE08E607
:105093001237AB1235FF1203466011400F7872E6E8
:1050A3002401796EF718E43619F780847874801533
:1050B300E4FEFF229083F3E0FEA3E0FF22F718E66D
:1050C30034FF19F722E62401FF18E436FE22E490A8
:1050D30083E3F0A3F0C21DC21EC21FC219FFFEFD6F
:1050E300FC9083CF11F99083D3120A079083D7746E
:1050F300FFF0E4A3F022120A07E4FFFEFDFC2231D5
:1051030023C21BC21CC21AFFFEFDFC90844211F98C
:10511300908446120A0790844A74FFF0E4A3F022B5
:10512300E490844CF0A3F02212293B9083D8E0FF53
:105133008F2812293BE528540F14B40700503B90E5
:1051430051491247D87302515E02516002516702FE
:105153005169025170025177025177800090837137
:105163007443F02280009083717454F02290837111
:105173007444F0229083717457F0221246675003EF
:10518300200267ED606414B40700505E90519612DC
:1051930047D8730251AB0251B40251BD0251DD0233
:1051A30051C20251CB0251D4908429E0FD7F01808A
:1051B30030908429E0FD7F02802712478680229069
:1051C3008429E0FD7F038019908429E0FD7F068018
:1051D30010908429E0FD7F078007908429E0FD7FFC
:1051E30005122B8B122FE4122C4D2220116A201052
:1051F30067908305E07002A3E0605D30131D908427
:105203002BE0C394195007E004F0D2098006908480
:105213002B7403F0C21320021F801630141A9084DB
:105223002BE0D394034005E014F0D209C21420020A
:1052330007E4FD7F13122B8B12293B752FFF75306B
:10524300127531BE7532FF7533127534C612478E2F
:10525300122DB0122CE880932220114A201047907F
:105263008305E07002A3E0603DA21472135015A2FF
:1052730001B39201D209C213C214200207E4FD7FD5
:1052830013122B8B12293B20010B752FFF75301244
:105293007531E48009752FFF7530127531ED122DCC
:1052A300B2122CE880B32212293B301102614A303A
:1052B3001002614A908305E07002A3E07002614A24
:1052C30030131C908429E0C394034004E4F0800667
:1052D300908429E004F0D209C213200227801E30F3
:1052E3001422908429E0D3940050057403F08006BF
:1052F300908429E014F0D209C214200207E4FD7F50
:1053030013122B8B908429E014601514601D146014
:10531300252403702D752FFF7530127531F6801F0C
:10532300752FFF7530127531FF8014752FFF75309F
:10533300137531088009752FFF75301375311112FC
:105343002DB2122CE841AD22E47855F630110261FA
:10535300EF30100261EF908305E07002A3E070026A
:1053630061EF30131F908423E0C36480948C500753
:10537300E004F0D209800690842374F4F0C2132071
:1053830002298020301424908423E0D36480947411
:105393004007E014F0D2098006908423740CF0C215
:1053A30014200207E4FD7F13122B8B12293B9084F8
:1053B30023E0FFC364809480400F7855EFF6752F88
:1053C300FF75301375311A8012908423E0F404784A
:1053D30055F6752FFF7530137531287532FF753308
:1053E30013753424122DB0122CE8614F2220114A78
:1053F300201047908305E07002A3E0603DA2137282
:10540300145015A202B39202D209C214C21320028D
:1054130007E4FD7F13122B8B12293B30020B752FF0
:10542300FF7530137531328009752FFF7530137591
:10543300313B122DB2122CE880B32253070FEFD366
:105443009409EF50042430FF222437FF225307F03E
:10545300EFC4540FFFD39409EF50042430FF2224E8
:1054630037FF22785D76FA30B708785D16E670F775
:10547300FF220000C2B57F0122908437E0D394005D
:1054830090843E40077404F0919680037403F07592
:10549300EAB022D19553EADF22F1A9A3E054607068
:1054A3001BA3E024FB600E14600E24FD600C240893
:1054B300700A02002602002E800680BD43EA4022C5
:1054C300908438E024FE602214602D24E260561498
:1054D300606324217078D13E741CF0A37466F0904D
:1054E3008433E4F0A37412F08068D13E741CF0A3FB
:1054F3007482F0901C848039908437E075F003A4A3
:10550300240BF582E5F0341DF583E493FB740193DA
:10551300FA740293F990843FEBF0A3EAF0A3E9F065
:10552300120768801ED13E741CF0A37479F0901C9E
:1055330078E493800ED13E741CF0A374A7F0901C02
:10554300A6E493FF908433E4F0A3EFF0800443EAEE
:10555300402290843CE0FE90843BE0FDEDFF7881A7
:10556300EEF6FE08EFF6908433E0FCA3E0FDC3D132
:10557300577F0050027F01908432EFF07881123719
:10558300B4EDD1574006A3EEF0A3EFF053EA7F90BA
:10559300843FA3E0FAA3E0F9EA497002C13890849A
:1055A30033E0FEA3E0FF4E7006D14EF5EA807A7831
:1055B30085EEF608EFF6D3D1464006187600087656
:1055C30008D14EFF7886E64FF5EAE47883F608F6CD
:1055D300C37984E778869618E66480F819E76480CF
:1055E30098501F90843FE0FBA3E475F00112085D1F
:1055F300A9F0FA120768F5E7788406E61870010641
:1056030080CE7885E6FE08E6FFC3908434E09FFDF4
:10561300908433E09EFCF0A3EDF04C70159084323F
:10562300E06006C3EFD146500990843FE4F0A3F055
:10563300A3F07F012275EA907F002290843F74FFDC
:10564300F0A3229408EE6480948022E5EA648054F7
:10565300804430229FEE6480F8EC648098228B486B
:105663008A49894AD3ED9408EC6480948040047C91
:10567300007D08D14E4DF5EAED1DAE0470011C4EC0
:10568300600FF1A07002054914F9120768F5E7806D
:10569300E722788176000876077890E690839EF07B
:1056A300C3742496FFE41896FED374079FEE6480B8
:1056B300F874809840077881EEF608EFF67881E673
:1056C300FE08E6FF788FE6FC08E62407F974823CBF
:1056D300FA7B01789F7C83F1987A83799E754D00DC
:1056E300754E087F017E00F10D7881E6FE08E678AD
:1056F3008F0826FFF618EE36FEF6C3EF9424EE6409
:105703008094804004E4F608F6228E488F498B4A41
:105713008A4B894C43EB28E549640145487006F1FF
:105723008C4002800CE54964024548700AF18C40C4
:1057330006754D00754E08E47883F608F6C3788441
:10574300E6954EE54D6480F5F018E6648095F050DB
:105753001CAB4A054CE54CAA4B7002054B14F912DD
:105763000768F5E60806E61870010680D0E5EB64E5
:105773008054804420FFE549640245487E0070025E
:105783007E40EF4E454EF5EB22D3E54E9408E54DB2
:1057930064809480227D011207427B0122AB48057D
:1057A3004AE54AAA492290843FE4F0A3F0A3F0908B
:1057B3008433F0A3F022B192EF7022908436E0B4E8
:1057C3000515A3E0FF4480F5EEEF90843E60057479
:1057D30003F080037402F090843674FFF02275485E
:1057E30001754984754A35E5ED540F640860064335
:1057F300EA407F0022E47881F608F61257A070028F
:10580300054914F9E5EF1207AE788206E618700130
:10581300067882E66408184670E143ED807F012232
:105823008B4B8A4C894DE54F154FAC4E7002154E8C
:105833004C601D0FEFCCEECC70010E14F5828C83FF
:10584300E0FD11547002054C14F9ED1207AE80D639
:1058530022AB4B054DE54DAA4C22908083E060744A
:10586300B405089080817401F0802278017C807DEA
:10587300017B017A8079837E007F401207427E009C
:105883007F407D007B017A807941120A55908083A5
:10589300E024FD603224FD602514601914601B149C
:1058A300600924087029E4F5AE8017908000740124
:1058B300F0E4A3F02211D8E4800811E1800411D8A8
:1058C30011E1908001F02290808411EB122381E496
:1058D300FF1221D122908084E09000E0F02290809A
:1058E30085E09000E2F0E422E0FFA3E0FCA3E0FD0A
:1058F30022C0E0C0F0C083C082C0D075D018E5E8F4
:1059030030E111E5EA30E609E5ED5430600353EA8E
:10591300BF53E8FDE5E830E45743EA3853EADF9044
:1059230080C3E0FFC394405041C374409FFFC394BE
:1059330008500280027F08787EEFF69080C3E0244F
:10594300C45125EFFD7C0012566153E8EF787EE6E3
:10595300FF9080C3E02FF0C394404004512D80108A
:105963009080C3E0FF1221D180061257B953E8EFAC
:10597300E5E830E37CE5ED30E6171257E17880EF98
:10598300F653E8F7E6606A5141EF706512549C8064
:1059930060E5ED540F6054908082E0C39440504B17
:1059A300E5ED540F787EF6087600787EE6FF08E68C
:1059B300FEC39F5014908082E02E2483F582E4344A
:1059C30080F583E5EFF00680E163ED8053E8F7129D
:1059D3002139787EE6FF908082E02FF0C394404027
:1059E30010115D53EA9043EA20800663ED8053E88B
:1059F300F7E5E830E20612569553E8FBE5E830E0B8
:105A03000353E8FEE5E830E70353E87FE5E830E5D4
:105A13000653E8DF12281BD0D0D082D083D0F0D039
:105A2300E032F9E43480FA7B0122908081E0600265
:105A3300E4F0908001E06005E4FF1221D12290841C
:105A430035E0FEB4210DA3E0B40908E4908082F0B0
:105A53007F0122EE64A17024908436E0B4011D53CB
:105A6300EA7F7B017A8079C47D087C0012566190BD
:105A730080C37408F0FF1221D17F01227F002251DD
:105A8300A450027E01EFD394017F0040027F01EF17
:105A93005E60037F01229083ACE07F0060027F01A0
:105AA300229083CDE0FFD394027E0022124FE4FFC5
:105AB300FEFDFC908379120A07E47858F6124682B9
:105AC300EF64016002616B202802615F51A4500200
:105AD3007E01EFD394017F0040027F01EF5E7002ED
:105AE30061781231BA717D7C007D321207C0717DFD
:105AF300C394D0EE94077F0040027F017856E6FC02
:105B030008E6FDC394E4EC940C7E0050027E01EEA3
:105B13005F6006785876038038C3ED94E4EC940C08
:105B23007F0040027F01718550027E01EE5F6006B7
:105B330078587602801BD3ED94CEEC94317F0050DD
:105B4300027F01718540027E01EE5F600C7858761A
:105B5300049083AC74FAF0801CE480169083ACE06C
:105B630060139083C5E0800A9083ACE06007908364
:105B7300C5E07858F67858E6FF227856EEF608EF37
:105B8300F622C3ED9488EC94137E0022124FE43086
:105B930028231247CEC39F25E0F6E418F67856E68D
:105BA300FFC3940A500FEF9017EB93C30896500569
:105BB30078560680E89083CEE0FF7856E6FED39FC2
:105BC3004006E02402F0800DEEC39F50089083CE80
:105BD300E014F080009083CEE0FFD3940A40057474
:105BE3000AF08008EF70059083CE04F09083CEE036
:105BF300FF22E4788B914AEF2403788CF6E43E1875
:105C0300F6EF24FDFFEE34FFFE788DF608EFF6C3C2
:105C13009083CB912E400F788B1237B4A3912E50E3
:105C23000591367F012291367F0022E09F9083CA3F
:105C3300E09E229083AFE0FFA3E09083CACFF0A35E
:105C4300EFF022F608F608F608F608F608F6223012
:105C53002A6112293BE4FD202B097F1C122B8BD2D6
:105C63002B80057F20122B8B908371744CF0A374CF
:105C730061F0A37473F0A37465F0A37472F090835E
:105C8300ABE024FC601F240424FA500A24F8500CCF
:105C930024F95011800F91BF7420800B91BFF0A3A2
:105CA3007420F0800591BFF0A3F0122CE8122FE4CA
:105CB300122C4D9083A8E0700291C72290837674D2
:105CC3003EF0A322C22AE49083BFF0A3F09083A600
:105CD300F0A3F09083ABF0C22B22E0FEA3E0FFE43D
:105CE300FCFD7B107A0EF9F8120873E40203C4C3B7
:105CF300EF9BFFEE9AFEED99FDEC98FC785D12099F
:105D0300FB785D1209C2E41203C4E4FBFA797A78E2
:105D1300441202A9E4FBFA79707842227855E6FE30
:105D230008E690E0002278591209C2E41203C4E4A1
:105D3300FBFA796178452275F00AA4FFAEF0785436
:105D4300EEF608EFF64E22120A07E47B107A27F9E3
:105D5300F822908422E0FCE41203CE7B857AEB796F
:105D6300C7783D0201A0122C4DD295D225C224E45E
:105D73009083C6F0A3F022908331120A07908452D5
:105D8300227D167F207E03122B0A78541209FBE42E
:105D930022F52F8E2E8D2D8C2C908423E0F53090C0
:105DA3008409227FA07E867D017C0078591209DE5A
:105DB300020873907FFFE493FFC4540FF535EF544B
:105DC3000FF53622E4FFFEFDFC785422E4FFFEFDCE
:105DD300FC90831C020A071202A912040290846138
:105DE300EEF0A3EFF02278551209FB7BA07A8679B7
:105DF300017800227889EEF608EFF67887A6060880
:105E0300F62275F00AEB120A13EA2208E6FE08E608
:105E1300FFC3785596EE189622786D1209FB7C84A1
:105E23007D4EAF2CAE2B22E6FE08E6FF7C017D689B
:105E33000208271209DED302099EEAFFC3E52D9F5C
:105E4300FFE49400FE22908459E09F908458E09EE2
:105E530022908458E0F535A3E0F53622FAA9827B37
:105E6300FF78D97C83221202A990845A020A07E0A0
:105E7300FF7E00C37480948022E52C2408F582E41D
:105E8300352B22E0FCFB5420FA53038022E0FD541F
:105E930020FCED5480FA22AF2CAE2BAD2AAC292284
:105EA300AF30AE2FAD2EAC2D22908388EEF0A3EF52
:105EB300F022122CE8908429E0FD221208FE785982
:105EC3000209FB7BDC7A0F794978402275F00AEDF1
:105ED300120A13EC22908456E09083E1F0227E8331
:105EE3007FD97C847D4E227887A60608A607228464
:0F5EF300908410E5F0F022E4FBFA793478432232
:027FFE00103A37
:00000001FF
